:020000040000FA
:100000006CEF05F0D9CFE5FFE1CFD9FF00C0E5FFE8
:1000100001C0E5FF02C0E5FF03C0E5FF04C0E5FF46
:1000200005C0E5FF06C0E5FF07C0E5FF08C0E5FF26
:1000300009C0E5FF0AC0E5FF0BC0E5FF0CC0E5FF06
:100040000DC0E5FF0EC0E5FF020EDBCF00F0030E92
:10005000DBCF01F0040EDBCF02F0050EDBCF03F0A7
:10006000060EDBCF04F000500110D8A4EAD002C085
:10007000E9FF03C0F3FF045031EC05F0056EF3CF48
:1000800006F00650E56E0550E56E000EE56E020EB8
:10009000E56EA5EC03F0076EF3CF08F0040EE12641
:1000A000096A0A6A400E07264B0E08224C0E0922E6
:1000B000000E0A2205C00BF006C00CF00D6A0E6A95
:1000C0000E50E56E0D50E56E0C50E56E0B50E56E72
:1000D0000A50E56E0950E56E0850E56E0750E56E72
:1000E0006AEC01F0076EF3CF08F0F4CF09F0E9CF26
:1000F0000AF0080EE126000EE56E000EE56E000E19
:10010000E56E040EE56E0A50E56E0950E56E085086
:10011000E56E0750E56E6AEC01F0076EF3CF08F06C
:10012000F4CF09F0E9CF0AF0080EE126FF0E07260A
:10013000FF0E0822FF0E0922FF0E0A220A50800F2E
:10014000800F08E1000E095C05E1010E085C02E188
:10015000000E075C0AE20850E56E0750E56E3C0EA3
:1001600041EC04F0020EE12664D00650E56E055025
:10017000E56E000EE56E080EE56EA5EC03F0056E6B
:10018000F3CF06F0040EE126096A0A6A400E05263E
:100190004B0E06224C0E0922000E0A220E50E56E6E
:1001A0000D50E56E0C50E56E0B50E56E0A50E56E95
:1001B0000950E56E0650E56E0550E56E6AEC01F0FB
:1001C000056EF3CF06F0F4CF09F0E9CF0AF0080E80
:1001D000E126000EE56E000EE56E000EE56E100ED7
:1001E000E56E0A50E56E0950E56E0650E56E055065
:1001F000E56E6AEC01F0056EF3CF06F0F4CF09F07E
:10020000E9CF0AF0080EE126FF0E0526FF0E0622B2
:10021000FF0E0922FF0E0A220550076E0650086ED7
:100220000850E56E0750E56E2C0E41EC04F0020E0E
:10023000E1260D0E78EC05F0AB8EAB88F36A010E6B
:1002400028D00050010A02E1015001E020D0040E44
:100250000226000E0322000E042202C0E9FF03C0A2
:10026000F3FF04505BEC05F0026E025007E0949A35
:1002700094889496C76A210EC66E06D0949A948884
:100280009486C76A250EC66EF36A010E02D0F36A21
:10029000E86AE4CF0EF0E4CF0DF0E4CF0CF0E4CF49
:1002A0000BF0E4CF0AF0E4CF09F0E4CF08F0E4CF9C
:1002B00007F0E4CF06F0E4CF05F0E4CF04F0E4CF9C
:1002C00003F0E4CF02F0E4CF01F0E4CF00F0E4CF9C
:1002D000D9FF1200D9CFE5FFE1CFD9FF00C0E5FF7C
:1002E00001C0E5FF02C0E5FF03C0E5FF04C0E5FF74
:1002F00005C0E5FF06C0E5FF07C0E5FF08C0E5FF54
:1003000009C0E5FF0AC0E5FF0BC0E5FF0CC0E5FF33
:100310000DC0E5FF020EDBCF00F0030EDBCF01F0D6
:10032000040EDBCF02F0050EDBCF03F0060EDBCFB1
:1003300004F0070EDBCF05F0080EDBCF06F0090E48
:10034000DBCF07F0D88003AED890086A0836085093
:100350000FE0031C0C6E021C0B6E011C0A6E001CCD
:10036000096E092A0DE10A2A0BE10B4A0C2A08D072
:1003700000C009F001C00AF002C00BF003C00CF08D
:1003800009C000F00AC001F00BC002F00CC003F07D
:10039000D88007AED890096A093609500FE0071CCB
:1003A0000D6E061C0C6E051C0B6E041C0A6E0A2AD0
:1003B0000DE10B2A0BE10C4A0D2A08D004C00AF00B
:1003C00005C00BF006C00CF007C00DF00D50E56E37
:1003D0000C50E56E0B50E56E0A50E56E0350E56E6D
:1003E0000250E56E0150E56E0050E56E41EC02F002
:1003F000006EF3CF01F0F4CF02F0E9CF03F0080E66
:10040000E1260950081A085016E0031C076E021C6A
:10041000066E011C056E001C046E042A04E1052A08
:1004200002E1064A072A07C0E9FF06C0F4FF05C03B
:10043000F3FF045007D003C0E9FF02C0F4FF01C07E
:10044000F3FF0050E4CF0DF0E4CF0CF0E4CF0BF05D
:10045000E4CF0AF0E4CF09F0E4CF08F0E4CF07F0EE
:10046000E4CF06F0E4CF05F0E4CF04F0E4CF03F0EE
:10047000E4CF02F0E4CF01F0E4CF00F0E4CFD9FF05
:100480001200D9CFE5FFE1CFD9FF00C0E5FF01C0E1
:10049000E5FF02C0E5FF03C0E5FF04C0E5FF05C0BE
:1004A000E5FF06C0E5FF07C0E5FF08C0E5FF09C09E
:1004B000E5FF0AC0E5FF0BC0E5FF0CC0E5FF0DC07E
:1004C000E5FF020EDBCF00F0030EDBCF01F0040EE0
:1004D000DBCF02F0050EDBCF03F0060EDBCF04F01E
:1004E000070EDBCF05F0080EDBCF06F0090EDBCFE1
:1004F00007F0086A096A0A6A0B6A200E0C6E034448
:10050000010B0D6E010E0D1600500026013602364D
:1005100003360850082609360A360B360D50D8A483
:10052000088007500B5C08E106500A5C05E10550A5
:10053000095C02E10450085C09E30450085E0550C0
:10054000095A06500A5A07500B5A00800C2ED7D76A
:1005500003C0E9FF02C0F4FF01C0F3FF0050E4CF85
:100560000DF0E4CF0CF0E4CF0BF0E4CF0AF0E4CFD1
:1005700009F0E4CF08F0E4CF07F0E4CF06F0E4CFD1
:1005800005F0E4CF04F0E4CF03F0E4CF02F0E4CFD1
:1005900001F0E4CF00F0E4CFD9FF1200D9CFE5FF9E
:1005A000E1CFD9FF00C0E5FF01C0E5FF02C0E5FFD4
:1005B00003C0E5FF04C0E5FF05C0E5FF06C0E5FF99
:1005C00007C0E5FF08C0E5FF09C0E5FF0AC0E5FF79
:1005D0000BC0E5FF020EDBCF00F0030EDBCF01F016
:1005E000040EDBCF02F0050EDBCF03F0060EDBCFEF
:1005F00004F0070EDBCF05F0080EDBCF06F000504D
:10060000011006E00050010A02E1015001E02DD086
:10061000076A086A0850800FF36E0650800FF35C7B
:1006200002E10550075C21E207500224096E0850E0
:1006300003200A6EE86A08BEE86804200B6E09C051
:10064000E9FF0AC0F3FF0B505BEC05F0096E09509F
:10065000E56E0150E56E0050E56E84EC04F0030E8B
:10066000E126072AD8B0082AD5D7E4CF0BF0E4CF8B
:100670000AF0E4CF09F0E4CF08F0E4CF07F0E4CFCC
:1006800006F0E4CF05F0E4CF04F0E4CF03F0E4CFCC
:1006900002F0E4CF01F0E4CF00F0E4CFD9FF120084
:1006A00093928A920001646B000E016E600E006EE0
:1006B000800E026E0250E56E0150E56E0050E56E50
:1006C000000EE56E010EE56E02EC00F0050EE1266F
:1006D000006A016A026A010E036E046A000EE56E8A
:1006E000010EE56EE4EC04F0056E020EE126055005
:1006F00009E0000EE56E010EE56EB7EC04F0020EA7
:10070000E126002A0150980A03E102503A0A01E06A
:100710000AD00050E56E000EE56E010EE56E84EC29
:1007200004F0030EE126012AD8B0022A032AD8B029
:10073000042A0450800F460F02E1990E035C02E385
:100740008A82CCD78A92CAD71200D9CFE5FFE1CFEF
:10075000D9FF00C0E5FF01C0E5FF02C0E5FF03C00F
:10076000E5FF020EDBCF00F0030EDBCF01F0040E3D
:10077000DBCF02F0050EDBCF03F000500001666F07
:100780000150676F02500001686F0350696F0001EC
:10079000665100016803F3CF00F0F4CF01F0005080
:1007A00000016A6F01506B6F00016651000169031F
:1007B000F3CF00F00001675100016803F3CF01F0AF
:1007C0000150002600016B51002600506B6F6BC07A
:1007D000F3FF6A51E4CF03F0E4CF02F0E4CF01F07D
:1007E000E4CF00F0E4CFD9FF1200000EF66E0B0E3E
:1007F000F76E000EF86E0900F550056E0900F55011
:10080000066E055002E106503BE00900F550006E0F
:100810000900F550016E0900F550026E090009004B
:10082000F550E96E0900F550EA6E0900090009006B
:10083000F550036E0900F550046E09000900F6CF6B
:1008400007F0F7CF08F0F8CF09F000C0F6FF01C0BD
:10085000F7FF02C0F8FF035002E1045007E009006F
:10086000F550EE6E0306F8E20406F9D707C0F6FF6E
:1008700008C0F7FF09C0F8FF0506C4E20606C5D7A1
:100880001200D9CFE5FFE1CFD9FF00C0E5FF01C0DD
:10089000E5FF02C0E5FF006E020EDBCF01F0030EA4
:1008A000DBCF02F0AC6AAB6A00B0AC8800A202D029
:1008B000AC8CAB8C00A401D0AC8E00A602D0AB886F
:1008C00001D0AB8A00A802D0AC8401D0AC949E9831
:1008D00000AC02D09D8A01D09D9A9E9A00AE02D0B3
:1008E0009D8801D09D980250B06E0150AF6E949CCF
:1008F000948EAC8AAB8EE4CF02F0E4CF01F0E4CF6B
:1009000000F0E4CFD9FF1200D9CFE5FFE1CFD9FF46
:1009100000C0E5FF01C0E5FF02C0E5FF03C0E5FF41
:10092000020EDBCF00F0030EDBCF01F0040EDBCFB5
:1009300002F00050011008E1025078EC05F087EC5D
:1009400005F0036E0350FBE10050010A02E1015083
:1009500001E002D002C0C9FFE4CF03F0E4CF02F00F
:10096000E4CF01F0E4CF00F0E4CFD9FF1200D9CFFB
:10097000E5FFE1CFD9FF00C0E5FF01C0E5FF02C000
:10098000E5FF020EDBCF00F0030EDBCF01F00050DD
:10099000011006E19E9A47EC05F0026E02500BD062
:1009A0000050010A02E1015001E004D0C7A002D0CA
:1009B000C95001D0E86AE4CF02F0E4CF01F0E4CFFF
:1009C00000F0E4CFD9FF1200D9CFE5FFE1CFD9FF86
:1009D00000C0E5FF01C0E5FF020EDBCF00F0030E13
:1009E000DBCF01F00050011006E19EAA02D0010EFB
:1009F0000FD0E86A0DD00050010A02E1015001E079
:100A000006D0C7A002D0010E03D0E86A01D0E86A80
:100A1000E4CF01F0E4CF00F0E4CFD9FF1200D9CF4A
:100A2000E5FFE1CFD9FF00C0E5FF01C0E5FF020E01
:100A3000DBCF00F0030EDBCF01F00050011009E125
:100A400087EC05F0006E005002E0E86A03D0010E6A
:100A500001D0E86AE4CF01F0E4CF00F0E4CFD9FFA1
:100A60001200E8AE06D0F3CFEAFFEE50EECFF3FF70
:100A70001200E8BC0BD0E9CFF6FFF3CFF7FFF86E1A
:100A80000900F5500900F5CFF3FF12001200F00E37
:100A900000016D156D6FABAC04D06D91ABA001D0B2
:100AA0006D81ABA402D000016D85ABA202D0000124
:100AB0006D87AE501200E8AE04D0F3CFEAFFEE50DF
:100AC0001200E8BC08D0E9CFF6FFF3CFF7FFF86ECD
:100AD0000900F5501200120017EEFFF027EEFFF0AC
:100AE000F86AA68EA69CF5EC03F050EC03F0FFD755
:100AF000ACAC04D0AC9000016DB3AC80AD6E120014
:100B00000100160B00006C00000001000000000E48
:080B1000ACA2010F120000006D
:020000040030CA
:0E000000FFF2FFFEFFFFBBFFFFFFFFFFFFFF52
:00000001FF
